:100000000C9439010C9456010C9471010C94560116
:100010000C9456010C9456010C9456010C94560104
:100020000C9456010C9456010C94A4180C9456018F
:100030000C9456010C9456010C9456010C945601E4
:100040000C9456010C9456010C9456010C945601D4
:100050000C945601FF04FF042B052B059305BE06E7
:10006000BE06BE06B1054A065B065B06E000E3007D
:10007000E2000000000000002C0000000000000072
:10008000E600E7006500E4000000E10064001D00F8
:100090001B00060019000500110010003600370093
:1000A0003800E50001510000390004001600070087
:1000B00009000A000B000D000E000F003300340091
:1000C0003100280000002B0014001A000800150061
:1000D00017001C0018000C00120013002F00300045
:1000E0003100000029001E001F0020002100220016
:1000F000230024002500260027002D002E003100BB
:100100002A000100010001000000000000000100C1
:1001100000000000000001000100010001000000DB
:1001200001000100010001000100010001000100C7
:1001300001000100010001000100010000000100B8
:1001400001000100010001000100010001000100A7
:100150000100010001000100010000000100010098
:100160000100010001000100010001000100010087
:1001700001000100010001000000C45CC05C01003E
:100180000100010001000100010001000100010067
:10019000010001000100005C09023B00020100A017
:1001A000FA09040000010301010009210101000115
:1001B0002240000705810308000109040100010332
:1001C000000000092101010001223200070583031C
:1001D0000800011201100100000008A0202D4200BB
:1001E00002010200010A0341007200650073000071
:1001F0000008034C0053004A0000000403090405F2
:10020000010980A101850319012AB700150126B74C
:1002100000950175108100C0050C0901A10185043C
:1002200019012AA002150126A0029501751081006E
:10023000C005010906A101050719E029E7150025F8
:10024000019508750181029501750881030507195B
:100250000029FF150026FF00950675088100050896
:100260001901290595057501910295017503910301
:10027000C00011241FBECFE5D8E0DEBFCDBF10E027
:10028000A0E6B0E0E0E3F9E302C005900D92A83EDD
:10029000B107D9F722E0A8EEB0E001C01D92A6395F
:1002A000B207E1F70E94B0120C94961C0C94000067
:1002B000A82FB92F80E090E041E050EA609530E04F
:1002C00009C02D9182279795879510F0842795274F
:1002D000305EC8F36F5FA8F30895EADF8D939D93B6
:1002E0000895CF93CFB7CF93C395839BE9F7839BB3
:1002F0000EC0839B0CC0839B0AC0839B08C0839B5A
:1003000006C0C0916D02C395C0936D02A6C0DF9375
:10031000C0916C02DD27CC58DD4F839B02C0DF917A
:10032000E6CF2F930F931F9300B32FEF03FB20F91A
:100330004F933F9310B34FEF012703FB21F93BE0AD
:1003400031C04E7F012F10B3216028C0102F4D7F88
:100350002260000000B329C04B7F2460012F000001
:1003600010B32BC010B3477F28602AC04F7E00B364
:1003700020612CC04F7D10B320622FC04F7B00B393
:10038000206432C0422700B349934FEF000010278A
:1003900013FB20F910B31C70C9F1297F91F20127DA
:1003A00003FB21F900B3237F89F2315058F1102764
:1003B00013FB22F910B3277E79F2012703FB23F9FF
:1003C0002F7C81F200B3102713FB24F92F7971F2EF
:1003D00000C010B3012703FB25F92F7359F200C0A9
:1003E00000B3102713FB26F9223040F200C010B3EF
:1003F000012703FB27F9243028F64F77206810B334
:100400000000F9CF10E81ABF00271CC03B503195FF
:10041000C31BD04010E81ABF0881033C11F10B3414
:1004200001F1209169021981110F1213EDCF4A8158
:10043000441F093669F10D3211F0013E29F74F7062
:1004400009F0042F009372023F914F911F910F9179
:100450002F91DF91CAB7C7FD47CFCF91CFBFCF91C3
:10046000189520917202222379F3109170021123C2
:1004700009F044C034300AF443C030937002209332
:100480006B0210916C023BE0311B30936C0238C060
:1004900000917002013094F50AE54F7049F43091F3
:1004A000710034FD2FC000937100C6E4D2E02EC06D
:1004B000433059F0443091F03091510234FD22C064
:1004C00000935102C2E5D2E021C030918A0234FD8E
:1004D00019C000938A02CBE8D2E018C030915D02C7
:1004E00034FD10C000935D02CEE5D2E00FC0279529
:1004F000A8F45150A9F4220F0000F9CF4AE503C037
:1005000042ED01C0432FC4E1D0E032E011B31C60E2
:10051000939A11BB02B320E41CE05F93012756E0DD
:1005200002BB279520F4515021F4220FF9CF012767
:1005300056E000003B5A02BBD0F2279528F45150F8
:1005400029F4220F0000F9CF012756E0279502BBBE
:1005500020F4515021F4220FF9CF012756E02991C0
:10056000332302BB21F6037F10917102110FC65194
:10057000D04002BB11F01093690210E81ABF086066
:1005800011B3137F402F437F5F9100C000C002BBB7
:1005900011BB42BB59CF81E0089581E008950C94CE
:1005A000CD0208950C94D1021F93CF93DF9300D016
:1005B00000D01F92CDB7DEB749835A836B83309149
:1005C000EB0089819A81311114C0662359F02223EE
:1005D00049F00E94F708182F682F89819A810E949C
:1005E000A00803C00E94CB08182F69817A81812F4F
:1005F00004C00E94F70869817A810F900F900F90D4
:100600000F900F90DF91CF911F910C942110FC015E
:10061000262F408151816281738184810C94D402A0
:1006200081E00895CF93DF93EC0160E00E9407031F
:10063000BE01DF91CF910C94D2020C9467110C94FF
:10064000631108950E944A070E9421032FEB87E25D
:1006500099E0215080409040E1F700C000000C94E8
:10066000CA180F931F93CF93DF938C0161E00E9410
:100670000703EC01B8010E94CF02882309F444C0AB
:10068000B801CE010E94AA138823F1F1B801CE016E
:100690000E945F178823C1F1B801CE010E948B141C
:1006A000882391F1B801CE010E94BB16882361F125
:1006B000F8018281882309F1CB358DE5D807C1F097
:1006C00050F4C115FCE5DF0781F0CF3DDC45A9F40E
:1006D0000E942E0E19C0CC35EDE5DE0761F0CD3558
:1006E000DD4559F40E94710D08C00E9422030CC020
:1006F0000E947A0D02C00E947D0DC801DF91CF914A
:100700001F910F910C94CB0280E0DF91CF911F914C
:100710000F9108950E944E1880E00E94DF130C9400
:10072000B5030E94CE120E94B8030C945418089589
:100730000C94970381E00895CF93C82F0E949A03E9
:10074000882329F0C1FF02C0919A01C09198CF91EE
:100750000895899A91980895CF93C82F0E9498037D
:100760008C2F0E949C03CF91089580E00C94AC03E1
:100770000E94BB170C94AC030E94BB179091EA0037
:10078000891721F08093EA000C94AC030895CF936D
:10079000DF93CDB7DEB72B970FB6F894DEBF0FBE51
:1007A000CDBF4F83588769877A878B8761110E94F5
:1007B000BD0C9E012F5F3F4F86E0F90111928A9593
:1007C000E9F785E0FE013796D90101900D928A95EF
:1007D000E1F789819A814C815D81452B31F09F3F02
:1007E00031F491E08F3F19F403C091E001C090E033
:1007F00090FF09C049815A816B817C818D819E81E6
:100800000E94DE0B05C0C9010E9410038111F2CFC6
:100810002B960FB6F894DEBF0FBECDBFDF91CF9100
:100820000895FC01808191810E9439090895CF9338
:10083000882309F44DC0C82F8CEF8C0F813AF8F44F
:100840008C2F0E947F16811143C06C2F8091620013
:10085000909163000E940A18882349F06C2F8091C0
:100860006200909163000E9442180E94DF0C6C2F7E
:1008700080916200909163000E9440180CC080E259
:100880008C0F883058F4C77081E001C0880FCA957A
:10089000EAF70E94A00CCF910C94DF0CEBE5EC0F73
:1008A000E33040F4F0E0E056FF4F808190E0CF91DC
:1008B0000C94D217C85AC73158F4EC2FF0E0EE0F61
:1008C000FF1FEE58FF4F80819181CF910C94E81764
:1008D000CF910895882349F1682F8CEF860F813AD4
:1008E00038F480916200909163000E9442180CC01D
:1008F00080E2860F883050F4677081E001C0880F75
:100900006A95EAF70E94A60C0C94DF0C8BE5860F23
:10091000833020F480E090E00C94D217685A67315D
:1009200020F480E090E00C94E81708951F93CF9393
:10093000DF93182FEB010E941704209741F087EBFB
:100940009BE00197F1F700C000002197F6CF812FBF
:10095000DF91CF911F910C946A04893319F060E004
:1009600070E002C060E570E00C949604882321F0EA
:100970000E94A00C0C94DF0C0895882321F00E94A3
:10098000A60C0C94DF0C0895CF92DF92EF92FF92A9
:100990000F931F93CF93DF937C01D62FC72FFC01BA
:1009A0001281058102950F700E94960C8823B9F080
:1009B0001123A9F08C2F807F803421F080E28D0FED
:1009C000883068F080912C0282FD09C082E00E948C
:1009D0003F0D0E94960C91E0D82ED92601C0D12C53
:1009E000CC2EC2948FE0C8228C2D90E08C309105E3
:1009F00008F0C4C1FC01E65DFF4F0C941B1C8C2F5A
:100A0000807FCF70882311F0C295C07F112399F0A9
:100A1000CC2309F49FC180E28D0F883010F0D111F2
:100A200004C08C2F0E94A00C03C08C2F0E94B00C1D
:100A30000E94DF0C8FC18D2F0E946A04CC2309F421
:100A40009DC180E28D0F883038F1DD2329F18C2F94
:100A50000E94B60C24C08C2F807FCF70803211F0A2
:100A6000C295C07FDD2319F0D130A1F13DC0809146
:100A70002C0282FF17C0112349F0CC2329F08C2FC0
:100A80000E94A00C0E94DF0C80E065C180E00E9403
:100A90006A04CC2309F472C18C2F0E94A60C0E9418
:100AA000DF0C6CC1112371F0002341F0013031F4EF
:100AB0000E94C00C8C2B0E94C80C60C10E94C00C0C
:100AC0008C2B1DC0002319F0013009F457C10E947E
:100AD000D50C25C0112321F0063008F04FC10EC0FF
:100AE000053008F04BC11BC0112361F0002331F029
:100AF000F701858180FF2EC18F7085838C2F0E9426
:100B0000B6043CC1002359F0D93309F034C1FFEFDA
:100B10000DEE12E0F15000401040E1F72AC18C2F99
:100B20000E94BD042BC18C2F86958695837019F089
:100B3000813061F023C1112321F08D2F9C2F937000
:100B400002C080E090E00E94D21720C1112321F062
:100B50008D2F9C2F937002C080E090E00E94E817D8
:100B600015C18C2F837009F047C011110BC12D2FB7
:100B7000229526952770220F220F6D2F6F70862FDA
:100B800090E0A0E0B0E0022E04C0880F991FAA1FD9
:100B9000BB1F0A94D2F7D4FF10C04FE050E060E0D2
:100BA00070E004C0440F551F661F771F2A95D2F7C7
:100BB000409550956095709503C040E050E0BA01B3
:100BC000C695C695C3708A019B01082B192B2A2B49
:100BD0003B2BC901B801C23049F058F4C13019F0BB
:100BE0000E94B607CFC00E94A407CCC00E94C807CD
:100BF000C9C00E94A207C6C0112319F08C2F8170B2
:100C000001C08695882309F4BDC02D2F2295269515
:100C10002770220F220F6D2F6F70862F90E0A0E0BB
:100C2000B0E0022E04C0880F991FAA1FBB1F0A94B0
:100C3000D2F7D4FF10C04FE050E060E070E004C095
:100C4000440F551F661F771F2A95D2F74095509580
:100C50006095709503C040E050E0BA01C695C69516
:100C6000C3708A019B01082B192B2A2B3B2BC9012E
:100C7000B801C23049F058F4C13019F00E947B0825
:100C800081C00E9469087EC00E948D087BC00E94BE
:100C9000DC0778C0CF70112339F08C2F0E94020836
:100CA0008D2F0E94B6046EC08D2F0E94BD048C2F24
:100CB0000E94230867C0D23F21F128F4D03F41F0C1
:100CC000D13FC1F043C0D33F19F1D43F79F03EC0CA
:100CD000112341F0053008F051C08C2F8F710E9414
:100CE00048084CC0063008F049C0F7CF80912C026C
:100CF00082FF18C0112339F08C2F8F710E940208D7
:100D00003DC01123C9F38C2F8F710E94230836C078
:100D1000112329F08C2F8F710E94ED072FC00E94A4
:100D2000E8072CC0112349F0CF718C2F0E940208D4
:100D300063E08C2F0E94240D21C081E00E943F0DB2
:100D40000230E0F082E00E943F0D18C0112331F024
:100D5000002391F28D2F0E94170410C0002399F2F6
:100D6000D93349F41FEF2DEE32E0115020403040CE
:100D7000E1F700C000008D2F0E946A0488EF8C0DFF
:100D8000843020F40E94BB170E94AC03DD20C9F020
:100D90000E94920C80FD15C0F70112820E948C0CFB
:100DA0000E940208C7010E9402070E948C0CDF917A
:100DB000CF911F910F91FF90EF90DF90CF900C9407
:100DC0002308DF91CF911F910F91FF90EF90DF905B
:100DD000CF9008950F931F93CF93DF93EC01688119
:100DE00079818A810E9444098C010E949F080E9497
:100DF0009007B801CE010E94C404DF91CF911F91EA
:100E00000F910895CF93DF93EC01988189812B8115
:100E10003C81232B31F08F3F31F481E09F3F19F467
:100E200003C081E001C080E080FD1DC0CE010E94B2
:100E30003103811110C00E94960C8823A1F08A8191
:100E4000882389F080912C0282FD0DC082E0DF9121
:100E5000CF910C943F0DCE010E94EA06CE01DF91A6
:100E6000CF910C941203DF91CF91089580E090E030
:100E70000E94D21780E090E00E94E8170E94BD0C0B
:100E80000C94DF0C80916200909163000E944418E2
:100E90000C9436070E94AD0C0C94420792959F70FB
:100EA000963079F010F4925001C09A50923068F464
:100EB000803F69F018F4883E40F409C0843F29F46B
:100EC00006C0883E20F0813F11F080E0089581E067
:100ED0000895FC01808191810E9439090E944E078A
:100EE0000895CF93DF9300D000D01F92CDB7DEB727
:100EF0000F900F900F900F900F90DF91CF9108956A
:100F0000CF93DF9300D000D000D0CDB7DEB72696C8
:100F10000FB6F894DEBF0FBECDBFDF91CF9108951D
:100F2000089508950C9491070C9492070E949407D9
:100F300060932201709323018093240190932501F3
:100F40000C9436070C9496070F931F93009122017F
:100F5000109123012091240130912501602B712BE8
:100F6000822B932B1F910F910C9496070F931F9335
:100F7000009122011091230120912401309125013B
:100F800060237123822393231F910F910C94960762
:100F90000F931F93009122011091230120912401AE
:100FA0003091250160277127822793271F910F9188
:100FB0000C9496070C9491070E94DA0760931E0127
:100FC00070931F0180932001909321010C943607A8
:100FD00060E070E0CB010C94DC070F931F9341E0BD
:100FE00050E060E070E08A019B0104C0000F111F17
:100FF000221F331F8A95D2F7C901B8011F910F91A3
:101000000C94DC070F931F9341E050E060E070E028
:1010100004C0440F551F661F771F8A95D2F7809131
:101020001E0190911F01A0912001B09121018A0120
:101030009B01082B192B2A2B3B2BC901B8011F91AF
:101040000F910C94DC070F931F9341E050E060E098
:1010500070E004C0440F551F661F771F8A95D2F7B2
:10106000409550956095709580911E0190911F015B
:10107000A0912001B09121018A019B01082319232D
:101080002A233B23C901B8011F910F910C94DC075F
:101090000F931F9341E050E060E070E004C0440F04
:1010A000551F661F771F8A95D2F780911E01909178
:1010B0001F01A0912001B09121018A019B01082705
:1010C00019272A273B27C901B8011F910F910C94BA
:1010D000DC070F931F9300911E0110911F012091B7
:1010E000200130912101602B712B822B932B1F91BA
:1010F0000F910C94DC070F931F9300911E01109128
:101100001F0120912001309121016023712382234E
:1011100093231F910F910C94DC070F931F93009161
:101120001E0110911F0120912001309121016027A3
:101130007127822793271F910F910C94DC07089544
:101140002FE0929F800D1124E82FE695E695E69515
:10115000877051E001C0550F8A95EAF785E0E89F56
:10116000F0011124E451FF4F20E030E070E04081B5
:10117000CB01022E02C0969587950A94E2F7817002
:10118000819584278523842781932F5F3F4F2530C6
:10119000310569F708952FE0929F800D1124682F83
:1011A000669566956695982F977085E0689FB00163
:1011B000112440E050E080E0FB01E40FF51FE45112
:1011C000FF4F208130E0092E02C0369527950A9402
:1011D000E2F721703327042E01C0220F0A94EAF7A8
:1011E000822B4F5F5F4F4530510531F70895BF9215
:1011F000CF92DF92EF92FF920F931F93CF93DF93E3
:101200008C01C0901E01D0901F01E0902001F09051
:1012100021018091220190912301A0912401B0919C
:101220002501C82AD92AEA2AFB2ACFE1D0E0D70132
:10123000C6010C2E04C0B695A795979587950A947C
:10124000D2F780FD04C0219790F7B12C07C0BC2EC7
:10125000B8018C2F0E9434100197A9F38B2DDF91D8
:10126000CF911F910F91FF90EF90DF90CF90BF90A3
:101270000895CF93DF93EC010E94F708BE010E940E
:101280003410DF91CF9108951F93CF93DF93EB013B
:101290009091EB00992321F0CB010E94390913C0F2
:1012A000882349F0CB010E94F708182F682FCE0140
:1012B0000E94A00804C0CB010E94CB08182FBE01D9
:1012C000812F0E943410DF91CF911F9108951F93B9
:1012D000CF93DF93C091260116E080912701C817B4
:1012E00099F0D0E01C9FF0011D9FF00D1124E85DE6
:1012F000FE4F4081518162817381848195810E947A
:1013000080072196C770E9CFDF91CF911F91089593
:10131000409158015091590160915A0170915B01BF
:1013200080915C0190915D010C948007EF92FF9297
:101330000F931F93CF93DF9380915D0182958F7000
:1013400009F065C080915A01882309F460C080913A
:101350002601F090270110915801009159016091E8
:101360005B0170915C0191E01F3F09F090E0C0913A
:101370006000D0916100292F96E0E92E8F1509F4C5
:1013800046C06115710521F00F3F21F030E003C028
:1013900031E001C0322F90E030FD36C0E89EF00110
:1013A000E99EF00D1124DF01A85DBE4F11963C911E
:1013B0001197301329C03C91311326C012963C91ED
:1013C0001297311121C013964D915C911497461BD1
:1013D000570B4C175D07C0F480915D018F708061E1
:1013E00080935D01E35DFE4F80818F70806180831B
:1013F00088E591E00E940207DF91CF911F910F9144
:10140000FF90EF900C94670901968770B7CFDF913A
:10141000CF911F910F91FF90EF9008959F92AF92FF
:10142000BF92CF92DF92EF92FF920F931F93CF93D1
:10143000DF93CDB7DEB761970FB6F894DEBF0FBE6E
:10144000CDBF8C0185E0F801DE011D9601900D9263
:101450008A95E1F7D8011296EC9090915801E091AD
:10146000590120915B0130915C012115310531F06A
:10147000EF3F31F481E09F3F19F403C081E001C0E8
:1014800080E0B82FB1709B2E80FD47C1D8014C91F0
:1014900011965C9111971396AD90BC90149788E5C6
:1014A000C82E81E0D82EF0905A01B501621B730B53
:1014B0002091600030916100FF2009F4D9C0809133
:1014C0005D016217730708F095C0282F207F09F08F
:1014D00052C05E1313C0491311C0FE2CE1100EC0A0
:1014E0008F70806180935D010E948809C6010E940F
:1014F000020780915D01F80185834DC1AB2831F071
:101500005F3F31F481E04F3F19F403C081E001C037
:1015100080E080FD03C081E08E2502C080E090E085
:10152000F82FF170FF2E80FF1CC0809126012091C2
:10153000270136E0821709F40BC190E0389FF001D3
:10154000399FF00D1124E85DFE4F6181561306C0EE
:101550006081461303C06281E61203C00196877062
:10156000E9CFFE2CEE2009F416C180915D01816067
:1015700080935D0154C05E1306C0491304C0E1109E
:1015800002C0F80199C0C8010E946907882361F16F
:10159000EE2051F120915D01822F82958F7090E0B5
:1015A000029774F0809158019091590198878F8328
:1015B0001986BB86AA862C87CE0107960E94020751
:1015C00086E0F801A8E5B1E001900D928A95E1F777
:1015D0000E9496090E9488090AC05E1711F1C8018D
:1015E0000E94690781112CC0C8010E940207FF24D4
:1015F000F394D1C0282F207F81F77A2DB98AA88A49
:101600006E2D89890E94710788E591E00E9402078A
:1016100086E0D6011D928A95E9F70E948809F12C8F
:10162000BAC04913DCCFE110DACFF8018583C801D5
:101630000E94020786E0D6011D928A95E9F7ABC0A9
:10164000EE2091F220915D01822F82958F7090E0C3
:1016500002970CF4B5CF80915801909159019A836B
:1016600089831B82BD82AC822E83CE010196A6CFD8
:101670006217730708F044C0FE2CEE2009F4B4CFC3
:101680005E1330C049132EC020915D0120FD21C0A2
:10169000822F82958F70482F50E041155105C9F077
:1016A000F80125834F30510541F08F5F982F9295B7
:1016B000907F822F8F70892B8583C8010E9402073B
:1016C00086E0F801A8E5B1E001900D928A95E1F776
:1016D0003CC086E0F801A8E5B1E001900D928A9542
:1016E000E1F759C0C8010E946907811169CF809153
:1016F0005D01816080935D01C8010E9402074BC0BB
:101700007A2DB98AA88A6E2D89890E94710786E090
:10171000D6011D928A95E9F718C0EE2009F464CF2E
:10172000C8010E946907F82E882309F45DCF86E07E
:10173000F801A8E5B1E001900D928A95E1F788E5FE
:1017400091E00E9411040E9496090E94880923C01A
:101750004D875E878D859E850E943909292F2295A8
:101760002F70223028F49F7039F0811105C00BC012
:10177000243028F49F7049F4805E883020F0C8013E
:101780000E9402079F2CF92C06C0D80115969C9147
:10179000907F91F7F8CF8F2D61960FB6F894DEBF4A
:1017A0000FBECDBFDF91CF911F910F91FF90EF90B2
:1017B000DF90CF90BF90AF909F9008951F93CF93ED
:1017C000DF93CDB7DEB72C970FB6F894DEBF0FBE10
:1017D000CDBF4F83588769877A878B879C87CE01D7
:1017E00007960E940E0A8823D1F09F8188852A855A
:1017F0003B85232B31F08F3F31F481E09F3F19F47B
:1018000003C081E001C080E080FD47C04F81588562
:1018100069857A858B859C850E9480073EC086E01D
:10182000FE013796DE01119601900D928A95E1F73F
:10183000FF81E8856A857B856115710531F0EF3F91
:1018400031F481E0FF3F19F403C081E001C080E082
:1018500080FD23C02091270130E0C90101968770E7
:1018600099274091260150E084179507F1F1F983FB
:10187000EA837D836C8396E0929FD001939FB00DA5
:101880001124A85DBE4FFE01319601900D929A95EC
:10189000E1F7809327010E94670916E080912601F5
:1018A00090912701891771F1189FC0011124885D5B
:1018B0009E4F0E940E0A882329F1E09126011E9F67
:1018C000F0011124E85DFE4F4081518162817381F6
:1018D000848195810E9480078091260190E0019685
:1018E0008770992780932601D9CF0E944A071092CA
:1018F000270110922601E8E5F1E086E0DF011D9264
:101900008A95E9F72C960FB6F894DEBF0FBECDBFCF
:10191000DF91CF911F9108958091660185958595FE
:10192000859508958091660187700895909166016C
:10193000977081E009F480E0089580917101089525
:1019400090917101892B80937101089580959091F8
:101950007101892380937101089510927101089596
:1019600090917001892B80937001089580959091DA
:101970007001892380937001089510927001089579
:1019800080916701089508950C94C30C0C94C40CC5
:1019900090912C0292FD08C090916701981721F058
:1019A000809367010C94C60C089580916701882389
:1019B00029F01092670180E00C94C60C0895CF9333
:1019C000DF93E0916200F091630080917101808368
:1019D000E0916200F0916300908180917001892B09
:1019E000808380916701882381F0E0916200F0910B
:1019F00063009081892B80838091620090916300C5
:101A00000E94FE1781110E94D50CC0916200D091F6
:101A1000630048E050E06EE571E0CE010E943B1C9F
:101A2000892B69F088E0FE01AEE5B1E001900D92EE
:101A30008A95E1F7CE01DF91CF910C94C717DF9122
:101A4000CF9108950C94C30C90912C0292FD10C07C
:101A500098E0899F90011124262B209366010E9413
:101A60000208809166018595859585950C94220DD7
:101A70000C9402081092660180E00C94220D2091D3
:101A800066018095822380936601982F977099F460
:101A900030E0482F082E000C550B2417350759F05D
:101AA00090912C0292FD07C08595859585950E94A1
:101AB00023080C943A0D089590912C0292FB222752
:101AC00020F9281769F080FB92F990932C028091FD
:101AD0002B0290912C020E94AA0D82E00C943F0DE3
:101AE000089580912C0282FB882780F991E0892754
:101AF0000C945C0D81E00C945C0D80E00C945C0D0A
:101B00006FEF7FEF80E090E00C94731C80E090E03A
:101B10000E94501C21E0893E9E4F09F020E0822F58
:101B2000089582E090E00C94481C83E090E00C94CF
:101B3000481CCF9384E090E00E94481CC82F82E2AA
:101B400090E00E94481C2C2F30E0A901582BCA01BC
:101B5000CF910895CF93C92F682F84E090E00E9421
:101B6000561C6C2F82E290E0CF910C94561CAB0176
:101B7000BC018FE090E00C94671CAB01BC0183E1D9
:101B800090E00C94671C60E070E0CB010C94BD0DFC
:101B900060E070E0CB010E94B70D0C94C30D69EEBC
:101BA0007EEF80E090E00E94731C60E082E090E0B5
:101BB0000E94561C60E083E090E00E94561C109248
:101BC000220110922301109224011092250160E05D
:101BD00084E090E00E94561C60E082E290E00E9467
:101BE000561C60E085E090E00E94561C60E086E0B4
:101BF00090E00E94561C6FEF87E090E00E94561C18
:101C000040E050E0BA0188E090E00E94671C60E08C
:101C10008DE090E00E94561C40E050E0BA0188E15F
:101C200090E00E94671C60E087E190E00E94561CF3
:101C300040E050E0BA018CE190E00E94671C60E057
:101C400070E080E290E00E94731C40E050E0BA0136
:101C500088E190E00E94671C0C94C80D0C94CF0D95
:101C6000682F8EE090E00C94561C0E9489186093B7
:101C7000800170938101809382019093830160932E
:101C80007C0170937D0180937E0190937F01089584
:101C900084B7806884BF84B7806884BF089581E07A
:101CA00008950C944F0E08950C94530E0C94530EFB
:101CB0000C94560E0C94530E0C945A0E0C94530E16
:101CC0000E94480E80E191E10E94B1170E945E0ED1
:101CD0000C945C0E0E94540E0C94530E0E942A1118
:101CE0000E94A9030C947F140E9476180E940F1280
:101CF0000E946E0E0E94CE120C94580E5F926F924C
:101D00007F928F929F92AF92BF92CF92DF92EF928B
:101D1000FF920F931F93CF93DF93CDB7DEB72A9730
:101D20000FB6F894DEBF0FBECDBF0E942412C82E9E
:101D300081110E94350E32E7832E31E0932E00E0B0
:101D400010E0502E802F0E944E115C01F401619032
:101D500071904F016826792661147104B1F40F5F08
:101D60001F4F0530110569F78FEF89838A831B8226
:101D70000E947D188160782F9D838C8349815A81D0
:101D80006B818D810E94C7033AC08091840181FDDF
:101D90000E945711D12CEE24E394F12CC3018E2123
:101DA0009F21892B29F10E94510E8823A9F0DE8200
:101DB0005F82AE20BF2081E0AB2809F480E08887F5
:101DC0000E947D188160782F9A8789874E815F8174
:101DD00068858A850E94C703000F111FF801EE581D
:101DE000FE4F80819181E826F926F182E08207C0CA
:101DF000D394EE0CFF1CFFE0DF12D0CFB0CF81E018
:101E0000C11001C080E02A960FB6F894DEBF0FBE65
:101E1000CDBFDF91CF911F910F91FF90EF90DF9099
:101E2000CF90BF90AF909F908F907F906F905F907A
:101E300008950E947E0E0E947E140C94BC03CF93E2
:101E4000DF930E943910EC01811522E59207E8F535
:101E5000811531E5930708F0B6C0883E910528F555
:101E6000803E910508F0E9C0883A910570F4853A02
:101E7000910508F07AC08130910509F473C008F427
:101E8000D9C0049708F0D9C0D5C08F3B910508F0A0
:101E9000D1C0C85AD0E0CC0FDD1FCD55DF4F09901F
:101EA000D881C02DCE019464C9C0811540E5940746
:101EB00008F069C0811550E4950708F060C09A9554
:101EC00081159F4108F4B9C0B5C0811536E5930767
:101ED00028F5811545E5940708F092C0811554E571
:101EE000950708F087C0AC0143705527282F269529
:101EF0002695C115D34508F06CC081E090E002C082
:101F0000880F991F4A95E2F740E2249F900111241F
:101F1000EC01C22BD32BCE019C6890C081152AE521
:101F2000920780F4811539E5930708F072C0811596
:101F300048E5940708F47EC0D82FCC27CE01806FE7
:101F4000906A7CC090568115904208F073C08D2F26
:101F50008F710E94CD10DD27D0628F71AE01582B9A
:101F6000CA016CC081E090E069C0C55AD0E0CF5290
:101F7000DF4F8881C82FD0E0CE0190645FC0DF7052
:101F8000CE01906A5BC074E0969587957A95E1F7EB
:101F9000282F23703C2F337081E090E002C0880F1F
:101FA000991F3A95E2F79C68AC01522B9A019C2F3D
:101FB0009F709695969550E2959FE0011124C90176
:101FC0008C2B9D2B3BC0D82FCC27CE01816F906AE4
:101FD00035C081E090E002C0880F991F4A95E2F772
:101FE00050E2259F90011124EC01C22BD32BCE018E
:101FF0009A6824C0D82FCC27CE01846F906A1EC067
:102000000E94CD108F7190E0D82FCC27CE01906226
:1020100015C08F700E94CD1094E0D695C7959A9503
:10202000E1F7CF70D0E0DC2FCC27D0699E01282BC0
:10203000C90104C080E090E001C0CE01DF91CF91E2
:1020400008952BE4829FC0011124FC012FE0729FB0
:10205000E00DF11D1124E60FF11DEE0FFF1FE459F5
:10206000FF4F8591949108950E9421100E941F0FA7
:1020700008958238910569F1B0F48133910509F42E
:102080006DC048F48932910509F463C08A32910524
:1020900009F469C008958533910509F455C0893361
:1020A0009105B9F00895833E910569F138F4803EB9
:1020B0009105B1F0823E910509F10895863E9105A2
:1020C000A9F1873E9105B9F1843E910509F064C0FC
:1020D00023C020912B0220FD4FC021FD4DC008954B
:1020E00080912B0280FD44C080912C0280FF44C06F
:1020F00080912B0284FD42C083EE4DC080912B0263
:1021000082FF38C0F5CF80912B0282FD33C08091D1
:102110002C0280FD31C0ECCF80912C0281FF32C0B7
:1021200080912B0284FD2AC087EE35C080912B025E
:1021300083FF26C0F5CF80912B0283FD21C08091C3
:102140002C0281FD1FC0ECCF80912B0285FD1CC0AD
:102150001DC080912B0285FD19C016C080912B02F5
:1021600086FD16C017C080912B0286FD13C010C0DB
:1021700089E311C082EE0FC080EE0DC080E00BC07D
:1021800086EE09C084EE07C089E205C085E303C07E
:102190008AE201C081E390E0089590912B0292FFC2
:1021A0000DC0282F2871283019F4877F846006C05D
:1021B000282F2471243011F48B7F886093FF0DC089
:1021C000282F2871283119F4877E846106C0282FB2
:1021D0002471243111F48B7E886120912C0220FF20
:1021E0000DC0382F3871383019F4877F816006C0F0
:1021F000382F3171313011F48E7F886021FF0DC08E
:10220000282F2871283119F4877E816106C0282F74
:102210002171213111F48E7E886194FD877E0895AD
:1022200080E008950C94800D0E9424128FE295E7BF
:102230000197F1F700C000000E94241284E00E9480
:102240004E1180FF04C00E9412110C94CA18089508
:102250000C9414110E94860D811102C00E942E0E52
:102260000E94910D809384010E94990D90932C02FD
:1022700080932B020E9428110E94950D682F70E018
:1022800080E090E00E94A20760911E0170911F0102
:1022900080912001909121010C94DA07E82FF0E061
:1022A000EE0FFF1FE95CFD4F808191810895089535
:1022B00088E78A95F1F7089500C008950C945811A5
:1022C00008950C9460110C9461110C9460110C949D
:1022D0006511F894E82FE295EF70F0E031A9282F0E
:1022E0002F7081E090E001C0880F2A95EAF7982FBF
:1022F0009095932391AB92A9892B82AB7894089502
:102300000F931F93CF93DF93C3EED0E089918F3F5C
:1023100011F00E94691180E0C83ED807B9F7C4EDFA
:10232000D0E003EE10E089918F3F11F00E94691117
:102330000C171D07C1F7DF91CF911F910F910895E1
:10234000BF92CF92DF92EF92FF920F931F93CF93A2
:10235000DF938C01C62FD0E0CE018D519F4F6C01D1
:10236000FC0190819F3F09F450C0B62EF894E92FEC
:10237000E295EF70F0E081A99F7021E030E001C0AC
:10238000220F9A95EAF7822B81AB82A92095282308
:1023900022AB78940E945C11E4EDF0E043EE50E053
:1023A00021E030E0E12CF12C61916F3F89F0A62F04
:1023B000A295AF70B0E0D0968C9190E06F7002C0A3
:1023C000959587956A95E2F780FD02C0C90102C024
:1023D00080E090E0E82AF92A220F331F4E175F07AA
:1023E00019F7F60180818F3F11F00E94691161E0B9
:1023F000E114F10409F460E08B2D0E945E11CC0F12
:10240000DD1FC00FD11FF982E882DF91CF911F91AC
:102410000F91FF90EF90DF90CF90BF9008950E94B2
:1024200080118AE0E7E3F2E0DF01982F1D929A9590
:10243000E9F7EDE2F2E0DF011D928A95E9F785E028
:102440000E946F120C941D03FF920F931F93CF9362
:10245000DF93CDB7DEB72A970FB6F894DEBF0FBE75
:10246000CDBF8E010F5F1F4F8AE0F80111928A9550
:10247000E9F7F12C6F2DC8010E94A011F394F5E04B
:10248000FF12F8CF4AE050E0B8018DE292E00E94DE
:102490003B1CFF24F394009709F4F12C892B41F0A5
:1024A0008AE0F801ADE2B2E001900D928A95E1F781
:1024B0002F2D45E067E372E08DE292E00E947012FA
:1024C0000E941F038F2D2A960FB6F894DEBF0FBE11
:1024D000CDBFDF91CF911F910F91FF900895089587
:1024E000FF920F931F93CF93DF93F82E092F162F90
:1024F000D72FC42F222349F081E0809387010E94C7
:102500007D189093860180938501809187018823AF
:10251000D9F080918501909186010E9495180597C8
:1025200098F0EF2DF02FA12FBD2F80E090E04C2FE1
:1025300050E08417950734F4219131912D933D9308
:102540000196F7CF10928701DF91CF911F910F91E4
:10255000FF9008950E94DF180E94740E0C94F018EA
:102560000E946B180E94D8180E94600E0E94AA1246
:102570000E94FE180E946A0EFBCF86E090E00C9449
:10258000481C682F86E090E00C94561C8091410214
:1025900084708961809341020C94C1120E94860D5F
:1025A000811104C00E942E0E0E94C6120E94BD120C
:1025B00080934102282F26952695269530E02430D9
:1025C000310524F087708861809341028091410237
:1025D00080FF04C086958695869501C080E00C94A6
:1025E000DF1320914102822F869586958695482F8C
:1025F00050E04330510554F48F5F982F990F990F95
:10260000990F822F8770892B80934102809141021C
:102610008160809341020E94C1128091410286959F
:10262000869586950C94DF1380914102982F96959C
:1026300096959695A1F0915E990F990F990F8770D5
:10264000892B80934102887F91E009F490E080918A
:10265000410290FB80F9809341020E94C112809157
:1026600041028695869586950C94DF1380914102F0
:1026700080FD13C0816080934102813019F489E0AC
:1026800080934102809141020E94C11280914102D7
:102690008695869586950C94DF1308958091410266
:1026A00080FF08C08E7F809341020E94C11280E0AB
:1026B0000C94DF1308958091410280FD0C944E1319
:1026C0000C94361390914102892F869586958695B4
:1026D0008F5F8F719770843038F4880F880F880F60
:1026E000892B8093410202C0909341028091410264
:1026F000887F91E009F490E08091410290FB80F99D
:10270000809341020E94C112809141028695869574
:1027100086950C94DF13843008F083E09091410299
:102720009770282F220F220F220F922B9093410295
:10273000987F21E009F420E09091410220FB90F97C
:10274000909341020C94DF130E948B1380914102FD
:102750000C94C1129C01FB018281882349F12E3B1C
:10276000FCE53F07C9F040F42C3BECE53E0769F07F
:102770002D3B3C4561F00895203C9CE5390791F0E4
:1027800070F0213C3C4589F0089583E001C080E071
:102790000E94A41380E008950E941413FBCF0E94AE
:1027A000F112F8CF0E945B13F5CF0E946213F2CFB3
:1027B00081E008958C9A94980895949808958F9242
:1027C0009F92AF92BF92CF92DF92EF92FF920F93C0
:1027D0001F93CF93DF93C82F843040F4811107C03B
:1027E0008FB58F7D8FBD0E94DD1304C0C3E08FB510
:1027F00080628FBDA6B5B7B52C2F30E00E94211C9A
:1028000023E030E040E050E00E94F91B0027122F47
:10281000232F342F012F122F232F332786B597B55F
:102820006CE070E00E94E51B6017710730F0C80192
:1028300069E070E00E94E51B52C086B597B5E6B42A
:10284000F7B4E6B5F7B5C6E0D0E0BE010E94E51BDF
:10285000060F171F211D311D4801590185E0880C05
:10286000991CAA1CBB1C8A95D1F7C701BE010E9406
:10287000E51B6F01E12CF12CA7019601260F371FF4
:10288000411D511DC501B4010E94F91B69017A0166
:10289000E6B5F7B5CA01B9010E94D51B9B01AC0191
:1028A000DF010E94301C9B01AC01C701B6010E94F0
:1028B000D51BDC01CB012FE0B695A79597958795A1
:1028C0002A95D1F706B517B520E030E008171907AB
:1028D0002A073B0718F466B577B5CB01BC0179BD73
:1028E00068BDDF91CF911F910F91FF90EF90DF9026
:1028F000CF90BF90AF909F908F90089508950E94C1
:10290000DA1382E28FBD89E18EBD8FEF9FEF97BD15
:1029100086BD0C94CE12CF93DF93EC01FB01828134
:10292000882309F43CC1C430FDE5DF0760F4CB3FE8
:102930009CE5D90788F49E0122503C45243131059D
:1029400008F02EC109C0C236EDE5DE0729F0C63A0F
:10295000FDE5DF0709F024C10E94990D90932C0238
:1029600080932B02C1318CE5D80709F4C6C008F06A
:1029700042C0C930ECE5DE0709F49BC000F5C53064
:102980008CE5D80709F485C078F4C330ECE5DE07A0
:1029900009F478C008F07AC0C230DC4509F0F5C00F
:1029A00080912B028160EFC0C7309CE5D90709F404
:1029B00078C008F07AC080912B028061E4C0CD30ED
:1029C000FCE5DF0709F487C058F4CB309CE5D90754
:1029D00009F479C008F07BC080912B0288606FC039
:1029E000CF30FCE5DF0709F480C008F082C0809199
:1029F0002B02877FC8C0CE3F9CE5D90709F471C080
:102A000000F5C531FCE5DF0709F485C068F4C33182
:102A10009CE5D90709F475C008F095C00E944A07E3
:102A200080912B028F77AFC0CC3FFCE5DF07A9F187
:102A300008F054C0CB3FDC4509F0A7C080912C02C0
:102A400040C0C230EDE5DE0709F489C058F4C11575
:102A50008DE5D80709F45AC008F069C080912C02AE
:102A600082602FC0C236EDE5DE0709F47CC0C63AAD
:102A7000FDE5DF0709F481C0C330DD4509F085C0FD
:102A800080E06EC080912B0282607DC080912B021D
:102A900016C080912B02886076C080912C028260E3
:102AA0004FC080912B0280626EC080912B028064A7
:102AB0006AC00E944A0780912B02806864C08460CB
:102AC00062C081603DC080912B028E7F5CC080918E
:102AD0002B028D7F58C080912B0216C080912C0252
:102AE00018C080912C028D7F2BC080912B028F7E8D
:102AF0004AC080912B028F7D46C080912B028F7B34
:102B000042C080912B02877F8B7F3DC080912C0239
:102B10008D7F8E7F15C080912B0282FB222720F9AA
:102B200091E0922790FB82F990FB83F92CC0809171
:102B30002C02982F909591708E7F892B90FB81F9B4
:102B400080932C0222C00E944A0780912B0287FBAF
:102B5000222720F991E0922790FB87F914C081E0A9
:102B60000E94300E12C080912B0284FB222720F994
:102B700091E0922790FB84F906C080912B02982F58
:102B8000909590FB80F980932B0280912B0290917D
:102B90002C020E94AA0D0E944A0780E001C081E039
:102BA000DF91CF9108950F931F9341E050E060E0D3
:102BB00070E08A019B0104C0000F111F221F331F08
:102BC0008A95D2F7C901B8010E94A2071F910F91FF
:102BD0000C944A078B3109F468C058F58B3009F41E
:102BE00086C078F4863009F445C020F4853009F4B5
:102BF0004BC07FC0873009F44AC0883009F477C0E1
:102C000078C0803109F464C068F48E3009F071C076
:102C10008091840182FB222720F991E0922790FB8A
:102C200082F94CC0863109F462C0893109F45FC071
:102C300060C08A32E1F060F4873209F455C028F4AC
:102C40008E3108F456C08D5150C08932E9F051C020
:102C5000833450F48A3308F045C0853309F444C006
:102C6000883309F444C045C08334F1F142C00E9466
:102C70002E0E3DC080918401817F8E7F80938401E0
:102C800081E08093880108950E94220330C08091E2
:102C90008401982F9095917090FB80F98093840126
:102CA000911125C0897F877F10C08091840181FBAD
:102CB000222720F991E0922790FB81F980938401EB
:102CC0009923A9F0809184018160809384010FC0D1
:102CD0008091840183FB222720F991E0922790FBC9
:102CE00083F9ECCF895301C080E00E94D31581E0C5
:102CF000089580E0089580E008950C947B16CF93AA
:102D0000C82F80918801882319F0813031F02BC0C1
:102D10000E949D0C823249F504C00E949D0C8232B3
:102D200061F48C2F0E947D16811104C08C2F0E94AB
:102D3000EA1517C081E090E014C08C2F0E947B162A
:102D400081110EC0C43149F018F4CB3049F00FC0E6
:102D5000C93219F0C83321F00AC01092880107C0A7
:102D600081E0817006C01092880180E002C080E09E
:102D7000F8CFCF910895CF93DF9386319C4541F5ED
:102D8000EB010E949D0C982F8A8120916200309166
:102D90006300882379F09A7A81E009F480E08093D7
:102DA0008901911102C069E201C065E3C9010E9475
:102DB00040180AC080918901811102C069E201C0F6
:102DC00065E3C9010E9442180E94DF0C80E001C047
:102DD00081E0DF91CF9108950F931F93CF93DF93FD
:102DE000C42FD22FFC0182818823C9F040938C012B
:102DF0000E947D1890938B0180938A0180E28C0F52
:102E0000883008F057C0C77081E001C0880FCA95AC
:102E1000EAF7DF91CF911F910F910C94B604809146
:102E20008C01481330C080918A0190918B010E94DF
:102E30009518883C910538F510E21D0FCD17B9F0B3
:102E400080E28C0F883040F4C77081E001C0880FA9
:102E5000CA95EAF70E94BD04183028F581E09D2F3D
:102E6000977001C0880F9A95EAF70E94B604802FE8
:102E70000E94AD041830F0F4D77081E001C0880FD3
:102E8000DA95EAF70AC080E28C0F883098F4C770B0
:102E900081E001C0880FCA95EAF7DF91CF911F91B9
:102EA0000F910C94BD04802FDF91CF911F910F9152
:102EB0000C94AD04DF91CF911F910F9108950F9362
:102EC0009C01CB01243F4CE5340731F188F4293DC6
:102ED000FCE53F07D9F02A3D4CE5340779F1283D60
:102EE0003C45A9F506E221EE41EE68ED7CE52BC0FC
:102EF000263FFCE53F07E1F0A8F0273F3C4539F5C8
:102F000007E225EE46EE67EF7CE51DC007E225EE01
:102F100045EE69ED7CE517C006E221EE40EE64EF78
:102F20007CE511C007E225EE44EE65EF7CE50BC0C1
:102F300006E221EE42EE66EF7CE505C008E221E004
:102F400045EE6AED7CE50E94EC1680E008C0FC01CD
:102F50008281882319F010928C0101C081E00F91C9
:102F600008959093E9008093E8000895909392016A
:102F7000809391010895E0919101F0919201309731
:102F800021F00190F081E02D099480E00895E09116
:102F90009101F0919201309721F00280F381E02DB0
:102FA0000994089520918F013091900128173907D5
:102FB00071F09093900180938F01E0919101F091D5
:102FC0009201309721F00680F781E02D0994089551
:102FD00020918D0130918E012817390771F090935F
:102FE0008E0180938D01E0919101F09192013097D3
:102FF00021F00084F185E02D09940895FC013296BA
:1030000097E080E0915029F021912223D9F38F5F3E
:10301000F9CF0895662349F0FC0132960896219174
:10302000621729F0E817F907D1F780E0089581E0E9
:1030300008959C01FC0132969FEF80E04191461774
:1030400089F09F3F19F4411101C0982F8F5F86309E
:10305000A9F79F3F39F0F901E90FF11D97FDFA95A6
:103060006283089508959C012A5F3F4FFC014281CD
:10307000461301C01282019682179307B9F708958B
:103080000C9419180C943318029626E0FC01119246
:103090002A95E9F7089508950C944B180C944C1850
:1030A0000C944B180C944B180C944B18CF930E9413
:1030B00052180E9424120E945018C0E08C2F0E94C7
:1030C0004E11892B29F4CF5FC530C1F780E001C0D4
:1030D00081E0CF91089508958091950181110C941C
:1030E0008A0308950E944A070C9491038BE083BFE2
:1030F0008BEB8CBF82E089BF08952FB7F894809145
:10310000420290914302A0914402B09145022FBF28
:1031100008952FB7F8946091420270914302809114
:103120004402909145022FBF08959C014FB7F89437
:103130008091420290914302A0914402B0914502D5
:103140004FBF821B930B089578941F920F920FB676
:103150000F9211248F939F93AF93BF93809142025C
:1031600090914302A0914402B09145020196A11DA5
:10317000B11D8093420290934302A0934402B09306
:103180004502BF91AF919F918F910F900FBE0F900D
:103190001F90189560E081E090E00E94791C9CE00F
:1031A00088E10FB6F894A89581BD0FBE91BDFFCF01
:1031B0000E947D18909394018093930108950E943A
:1031C000BA1B8B9A80E0815041F0A895E7EBFBE0B9
:1031D0003197F1F700C00000F6CF8B9878940895EE
:1031E0000E94DD190E94B6172FEB84ED91E021506B
:1031F00080409040E1F700C00000089580916D028A
:10320000882389F010926D020E947D18909394019A
:1032100080939301809195018823D1F110929501BB
:103220000E94721811C080919501811111C0809186
:103230009301909194010E949518069728F081E0DF
:10324000809395010E946C1880919501882301F16B
:103250000E946C180E945618882339F1F89421B303
:10326000939A822F8C6081BB92B38CE0982792BB9B
:103270003FE54AEE90E0315040409040E1F700C019
:10328000000092B3892782BB21BB9398789408955C
:103290000E94C31A80917302882329F08091510201
:1032A00084FD0E94190F0C948419089580912A02BC
:1032B0000895089590919B01981307C0209199015A
:1032C00030919A0126173707A9F080939B017093DC
:1032D0009A0160939901809396017093980160938D
:1032E000970180918A0284FF05C063E086E991E03E
:1032F0000C94BF1A0895BC0184E00C945A19BC01C7
:1033000083E00C945A190895CF93DF93CAE0D0E07C
:103310008091510284FF18C08091A7019091A8016B
:103320009817E1F028E0829FC001112468E08755DA
:103330009E4F0E94BB1A8091A70190E001968F706A
:1033400099278093A7010AC00E94C31A87EB9BE0CC
:103350000197F1F700C000002197D1F6DF91CF91DE
:103360000895CF93DF93EC01A091A801B0E0CD01C7
:1033700001968F7099272091A701281779F093E083
:10338000AA0FBB1F9A95E1F7A755BE4F98E0FE0123
:1033900001900D929A95E1F78093A8010E94C31ABB
:1033A0000E94841988E0FE01AFE9B1E001900D921E
:1033B0008A95E1F7DF91CF91089584E690E0089532
:1033C000FC01808180768032A1F58181813061F4B9
:1033D00084819581892B69F58FE991E090936F0243
:1033E00080936E0288E00895823041F489E292E091
:1033F00090936F0280936E0281E008958A3021F4E9
:1034000083818093290215C0893099F48281938148
:103410008115924081F484819581892B61F481E04A
:1034200080939E018681978190939D0180939C015A
:1034300002C080E008958FEF089520919C013091A3
:103440009D01232B71F020919E01213051F4FC014C
:10345000808180932A0210929D0110929C0181E04C
:1034600008958FEF08950895FC0193819330D9F06A
:1034700068F4913081F0923009F059C088E991E008
:1034800090936F0280936E028BE30895913249F11D
:103490009232B9F14CC083ED91E090936F0280932A
:1034A0006E0282E108958281813099F050F082307D
:1034B000F1F585EE91E090936F0280936E028AE0C1
:1034C00008958BEF91E090936F0280936E0284E0F9
:1034D000089581EF91E090936F0280936E0288E0EF
:1034E00008958281882329F0813009F583EC91E0E9
:1034F00002C08AEA91E090936F0280936E0289E0A5
:10350000089584819581009751F0019781F48FEFA0
:1035100091E090936F0280936E0282E3089581E3BD
:1035200092E090936F0280936E0280E4089580E0B1
:1035300008951F93CF93DF93162FEA01288124FF6C
:1035400005C0398128E82327298302C02AE528837A
:10355000212FFC01CE010296DC0131913D932150D7
:103560001216DCF3612F0E946D011C5F1883DF913E
:10357000CF911F91089541E552E00C94991A4AE8C1
:1035800052E00C94991ACF93DF93609170026350CC
:1035900067FD93C080916C02CCE0D0E0C81BD109DC
:1035A000CC58DD4F80916B02803120F4CE010E9417
:1035B000331A81C08D3209F06EC0683009F07BC0CB
:1035C00083EC809346028AE58093710010926A0230
:1035D0008881807621F0CE010E94E01949C09A814D
:1035E00010924F028981811106C0109250022FE47F
:1035F00032E082E038C0853019F49093710230C017
:103600008630A1F48B81813041F0823031F08330FB
:1036100021F0813211F0823221F4CE010E94341A5D
:1036200001C080E090E490936A0222C0883089F063
:10363000893019F49093730213C08A3069F08B308B
:1036400079F48BE48093520280938B0280935E0224
:1036500007C023E732E002C02FE432E081E003C07C
:103660002FE432E080E030936F0220936E0209C0B5
:103670008F3F39F4988197FD8E8190E890936A028C
:1036800007C09F81911104C09E81981708F4892F6B
:103690008093700010C080916A0287FF0CC0CE0139
:1036A0000E941D1A8F3F21F48EE18093710003C0A8
:1036B000811110927000109270028091710084FF4D
:1036C0004CC0809170008F3F09F447C0C82F8930EB
:1036D00008F0C8E08C1B809370009091460288E847
:1036E000892780934602CC2359F180916E029091F4
:1036F0006F0220916A0226FF12C0A6E4B2E02C2FCE
:10370000AC0146545240FA01EA0FFB1FE4911196B6
:10371000EC931197215011962111F5CF08C0E7E4E1
:10372000F2E0DC012C2F3D9131932150E1F701961D
:103730002FEF2C0F820F911D90936F0280936E02DA
:103740006C2F87E492E00E946D01CC5FCC3019F0C1
:103750008FEF80937000C093710084E190B39C70F0
:1037600031F48150D9F71092710210926902DF9101
:10377000CF910895CF93DF9385B7886085BF8BB7CE
:1037800080688BBFC1E5D2E08BE48983AAE8B2E010
:1037900011968C931197EDE5F2E081838AE5888399
:1037A0008C938083DF91CF910895DB018F939F935A
:1037B0000E94301CBF91AF91A29F800D911DA39FCD
:1037C000900DB29F900D11240895AA1BBB1B51E1CF
:1037D00007C0AA1FBB1FA617B70710F0A61BB70B81
:1037E000881F991F5A95A9F780959095BC01CD0126
:1037F0000895A1E21A2EAA1BBB1BFD010DC0AA1F32
:10380000BB1FEE1FFF1FA217B307E407F50720F049
:10381000A21BB30BE40BF50B661F771F881F991FC4
:103820001A9469F760957095809590959B01AC010D
:10383000BD01CF010895EE0FFF1F0590F491E02D1B
:103840000994A29FB001B39FC001A39F700D811D79
:103850001124911DB29F700D811D1124911D089599
:103860000E94211CA59F900DB49F900DA49F800DD8
:10387000911D11240895FB01DC0104C08D9101907C
:10388000801921F441505040C8F7881B990B0895C6
:10389000E199FECF9FBB8EBBE09A99278DB3089527
:1038A000A8E1B0E042E050E00C94881C262FE1999A
:1038B000FECF9FBB8EBBE09A01970DB2021631F08E
:1038C0002DBB0FB6F894E29AE19A0FBE08950396C5
:1038D000272F0E94571C0E94561C252F0E94571C00
:1038E000242F0C94571C0196272F0E94571C0C94D0
:1038F000561C262FE199FECF9FBB8EBB2DBB0FB66A
:10390000F894E29AE19A0FBE01960895DC01CB018A
:10391000FC01E199FECF06C0FFBBEEBBE09A3196F9
:103920000DB20D9241505040B8F70895F894FFCF72
:10393000C80068015619B11983197F197B195919E3
:10394000FF5AE200E900EA00B500B600B700CD007A
:103950008301CC008A0192019401210223022402F6
:103960002502260227022A02B300B4006F0070006D
:10397000818283E200E900EA00B500B600B700CD1D
:10398000008301CC008A01920194012102230224C8
:10399000022502260227022A02B300B4006F00703B
:1039A000008182839091929394959697373635341F
:0839B0003332076061626364B9
:00000001FF
